:100000000C947B020C94BF020C94BF020C94BF02B0
:100010000C94BF020C94BF020C94BF020C94BF025C
:100020000C94BF020C94BF020C94630D0C94350E1B
:100030000C94BF020C94BF020C94BF020C94BF023C
:100040000C94BF020C943F220C94BF020C94BF028C
:100050000C94BF020C94D21B0C94BF020C94BF02F0
:100060000C94BF020C94BF020C94BF020C94BF020C
:100070000C94BF020C94BF020C94BF020C94BF02FC
:100080000C94BF020C94BF020C94BF020C94BF02EC
:100090000C94BF020C94BF020C94BF020C94BF02DC
:1000A0000C94BF020C94BF020C94BF02A20EC40EAB
:1000B000B20FC40EB20F090F2C0FB20F810F940FA5
:1000C0006312631292129212C812E81219141914D0
:1000D000F3121914A313A3130A14191419141314E3
:1000E000B013B013B013B013B013B013B013B013F8
:1000F000B013B013B013B013B013B013B013B013E8
:10010000C213CF13D613DD13E7130000F0A1F0A242
:1001100035002B002971E100C10000001E00140011
:1001200004421D71C200E1001F001A0016001B00EE
:10013000E104E300200008000700060050002C0046
:1001400021001500090019004F004D002200170082
:100150000A000500000065742F002D000000007FDC
:1001600000004A0030002E000000007700004B0025
:1001700023001C000B00110000002971240018004E
:100180000D00100052004E0025000C000E0036003D
:1001900051002800260012000F0037002F002B000E
:1001A00027001300330038713000E2002A003100CC
:1001B0003400E500C1000000010001000100010061
:1001C000010000003A001E0220022202010001008C
:1001D0003B001F0221022302010001003C002F020C
:1001E00026022F00010001003D00300227023000EE
:1001F000010001003E00310235003502000001001F
:1002000001000100000001000000010001000100E8
:1002100000000100000001003F00520051002402D4
:10022000000001004000240021001E000100010028
:100230004100250022001F00370001004200260077
:100240002300200027000100430025022E02310078
:100250002E000100440045000100010001000000E3
:100260000100010001000100010000000100010087
:100270000100010001000100010001000100010076
:100280000100010001000100010001000100010066
:100290000100010001000100010001000100010056
:1002A0000100010000000100010001000000010048
:1002B0000000010001000100000001000000010039
:1002C00001000100F2000100000001000100010036
:1002D000F1000100A90001000100F400F000AC00F1
:1002E000AA00B6000100F500F300AB00A800010071
:1002F00001000100010001000100010001000100F6
:10030000AE00010001000000160345007200670006
:100310006F0044006F007800200045005A00000084
:1003200016034500720067006F0044006F007800FC
:10033000200045005A0000000403090409026D0072
:10034000040100A0FA0904000001030101000921D1
:1003500011010001223F000705810308000A09047A
:1003600001000103010200092111010001224D00D9
:100370000705820308000A090402000103000000C7
:100380000921110100012236000705830308000A34
:1003900009040300010300000009211101000122EA
:1003A000390007058403100001120110010000004C
:1003B00008EDFE071301000102000105010906A175
:1003C00001050719E029E715002501950875018148
:1003D0000205081901290595057501910295017518
:1003E00003910105071900297715002501957875F6
:1003F000018102C005010980A101850216010026C4
:10040000B7001A01002AB700751095018100C005D8
:100410000C0901A1018503160100269C021A0100A6
:100420002A9C02751095018100C005010902A101F5
:100430000901A100050919012905150025019505E6
:1004400075018102950175038101050109300931AA
:100450001581257F95027508810609381581257F4C
:10046000950175088106050C0A38021581257F95CE
:100470000175088106C0C005010906A1010507191B
:10048000E029E715002501950875018102950175A0
:100490000881010508190129059505750191029545
:1004A00001750391010507190029FF150025FF9526
:1004B0000675088100C00000000000000000000078
:1004C00000010204060A0F17202C3A4A5D71879D2D
:1004D000B3C7DAE9F5FCFFFCF5E9DAC7B39D87712C
:1004E0005D4A3A2C20170F0A0604020100000000A2
:1004F00000000000000011241FBECFEFDAE0DEBFD5
:10050000CDBF04B603FE24C08091FB019091FC0195
:10051000A091FD01B091FE018730904BA740B04BF8
:10052000B9F41092FB011092FC011092FD0110929F
:10053000FE0114BE84B7877F84BF88E10FB6F894AC
:1005400080936000109260000FBEE0E0FFE3099529
:1005500011E0A0E0B1E0ECE0F8E402C005900D92FB
:10056000A433B107D9F711E0A4E3B1E001C01D92B3
:10057000AB3FB107E1F70E94A70A0C9404240C9446
:1005800000001092B9008AE08093B800089594EAC0
:100590009093BC009091BC0097FFFCCF9091B90064
:1005A000987F983021F0903111F081E00895809388
:1005B000BB0084E88093BC008091BC0087FFFCCF27
:1005C0008091B900887F883111F0803471F780E024
:1005D000089584E98093BC008091BC0084FDFCCF29
:1005E00008958093BB0084E88093BC008091BC0098
:1005F00087FFFCCF9091B900987F81E0983209F491
:1006000080E0089584E88093BC008091BC0087FF5F
:10061000FCCF8091BB00089580910101811115C02C
:1006200080E40E94C7028093010181110CC082E125
:100630000E94F10280930101811105C08FEF0E9499
:10064000F102809301010E94E90284B1807F84B9A4
:1006500085B1807F85B98AB1837F8AB98BB1837F69
:100660008BB93E98469808950E94C7048093010173
:100670000E940C0380B38C7080BB81B3836F81BBFD
:10068000A5E3B1E0E3E4F1E08EE08E0F11921D925C
:100690008E13FCCF0C94B104BF92CF92DF92EF92F5
:1006A000FF920F931F93CF93DF93809101018823D3
:1006B00079F0809134018F5F80933401811108C0FB
:1006C0000E94C70480930101811102C00E94590455
:1006D00005E311E0C0E0D0E0DD24D39482E0C82E31
:1006E000EE24E394F12CC730D10500F5809101018F
:1006F000811164C080E40E94C702809301018111CE
:1007000012C082E10E94F1028093010181110BC0AD
:10071000C7010C2E01C0880F0A94EAF780950E9449
:10072000F102809301010E94E90248C0CA30A1F0A1
:1007300028F4C83059F0C93061F005C0CC3089F0D8
:1007400070F0CD3089F0209A289810C0219A29980D
:100750000DC0229A2A980AC0239A2B9807C0529A51
:1007600001C0539A5B9802C03E9A469890EA9A95C7
:10077000F1F79FB1799902C082E001C080E09170E9
:100780009D25982B7C9902C084E001C080E0892BD4
:100790007D9902C038E001C030E0832B7E9902C011
:1007A00020E101C020E0822B9FB19095991F9927ED
:1007B000991F9295990F907E892B0FC0809101010E
:1007C000811149C080E40E94C702809301018823FF
:1007D00079F1B12C0E94E9028B2DF80190819817D4
:1007E00019F08083C09200010E940C0321960F5FD4
:1007F0001F4FCE30D10509F076CF809100018823BC
:1008000061F1815080930001882339F08FE99FE0E6
:100810000197F1F700C0000020C0A3E4B1E0E5E3D8
:10082000F1E0CF01825F91919D938E13FCCF15C0B3
:1008300083E10E94F102809301018111CACF81E41A
:100840000E94C702809301018111C3CF0E9402035D
:10085000B82EB094BFCF80E0C0CF0E94570481E093
:10086000DF91CF911F910F91FF90EF90DF90CF908C
:10087000BF900895E82FF0E0ED5BFE4F8081089572
:1008800008950F931F93CF93DF93C3E4D1E010E05B
:100890000C2F025F899190E00E94F81A180F0C1338
:1008A000F9CF812FDF91CF911F910F9108950C9473
:1008B000270556985E9825982D9826982E98279863
:1008C0002F988FEF90E09093890080938800909309
:1008D0008B0080938A0090938D0080938C00259AE2
:1008E0002D9A2FEF80E792E0215080409040E1F771
:1008F00000C00000269A2E9A2FEF80E792E0215048
:1009000080409040E1F700C00000279A2F9A2FEF17
:1009100080E792E0215080409040E1F700C0000065
:1009200025982D982FEF80E792E02150804090404D
:10093000E1F700C0000026982E982FEF80E792E0A4
:10094000215080409040E1F700C0000027982F9888
:1009500056985E9825982D9826982E9827982F9827
:10096000089589EA8093800089E08093810024982B
:100970002C983F988AB18F748AB96E98479A8BB138
:10098000806B8BB9769A0E9459040C94260580E2FC
:10099000809301018091510181110EC00E94C1021A
:1009A00081E0809351012FEF83ED90E3215080404F
:1009B0009040E1F700C0000080E40E94C7028093ED
:1009C000010181112EC00E94F10280930101811169
:1009D00028C00E94F10280930101811122C08FE39F
:1009E0000E94F1028093010181111BC00E94E90263
:1009F00080E40E94C70280930101811112C08CE043
:100A00000E94F1028093010181110BC00E94F1024A
:100A100080930101811105C08FE30E94F102809350
:100A200001010E94E90280910101089561110BC04A
:100A3000FC018281882321F085EE0E94071103C00A
:100A400085EE0E94CF1180E090E0089508956091B6
:100A5000BD017091BE018091BF019091C0010E94C3
:100A6000041B56985E9825982D9826982E982798BE
:100A70002F98813019F0823021F00895259A2D9A0F
:100A80000895269A2E9A089581E0089581E00895A8
:100A90000C94460508950F931F93CF93DF938C0119
:100AA000FC01C081D181CE010E947D19BE010E944E
:100AB000F405EC01B8010E944805882309F48DC0B3
:100AC000F8018281882309F44AC080915D01811177
:100AD0001FC0C431F0E5DF0709F051C00E944A058C
:100AE00081E080935D010E949C1B90935C01809348
:100AF0005B01109254011092560110925501109210
:100B000058011092570110925A011092590165C074
:100B100080915B0190915C010E94A81B883C91052B
:100B200070F480915401E82FF0E0EE0FFF1FEB5AB4
:100B3000FE4FD183C0838F5F809354014EC0C43871
:100B400080E5D80721F0C538D04501F13AC0F80159
:100B50008281882341F01092520182E01EC0C43885
:100B6000E0E5DE0759F580915201811106C086E269
:100B70000E94071186E20E94CF1182E01CC0C43897
:100B8000F0E5DF0741F3C538D045D9F4F80182819B
:100B9000882331F01092530180E20E941E121DC082
:100BA00080915301811106C087E20E94071187E2FC
:100BB0000E94CF1180E20E9425120FC0C538D04597
:100BC00029F381E08093520180935301C801DF91A2
:100BD000CF911F910F910C94440580E0DF91CF914C
:100BE0001F910F910895089596E0799FF0011124C7
:100BF00094E5899FE00DF11D1124E60FF11DEE0F24
:100C0000FF1FE05FFE4F859194910895880F991F13
:100C1000FC01E657F040859194910895880F991F43
:100C2000FC01E65FFE4F8591949108950F931F9309
:100C3000CF93DF93EC01811520E3920750F5C115A6
:100C400080E2D80708F0C3C0CB3BD10590F4C83A86
:100C5000D10508F06AC0C53AD10508F05BC0C430C0
:100C6000D10508F0D0C1219709F0CAC101E010E018
:100C70000AC2CF3FD10511F008F0C5C1C03FD10570
:100C800008F0A2C0CE01805E9109089708F4BBC1AC
:100C9000B7C1C13090E5D90709F4A2C020F5C03131
:100CA0008FE4D80770F4C11590E4D90708F094C018
:100CB000C11521E3D20708F0A3C1DD278E01106C16
:100CC000E2C1C115D04509F09BC10E9484148FEF89
:100CD00094E32CE0815090402040E1F700C00000F8
:100CE0000E94F71BD0C1C11597E5D90758F4C03150
:100CF00021E5D20708F01CC1C43180E5D80708F40B
:100D000075C07EC1CE0190578115904108F078C121
:100D1000DF7073C1C53AD10509F477C1C63AD10570
:100D200009F076C102E810E4AEC1C83AD10509F471
:100D300072C1C93AD10509F471C1CA3AD10509F4A1
:100D400070C1CB3AD10509F46FC1CC3AD10509F491
:100D50006EC1CD3AD10509F46DC1C03BD10509F48E
:100D60006CC1CE3AD10509F46BC1CF3AD10509F473
:100D70006AC1C13BD10509F469C1C23BD10509F47F
:100D800068C1C33BD10509F467C1C43BD10509F46F
:100D900066C1C53BD10509F465C1C63BD10509F45F
:100DA00064C1C73BD10509F463C1C83BD10509F44F
:100DB00062C1C93BD10509F461C1CA3BD10509F43F
:100DC00060C100E014E45FC18E0110655CC1CE011A
:100DD0009F700E940E0658C1DF708E01106A53C1C9
:100DE0008091DA0181608093DA014DC10E949C1DDF
:100DF000811102C00E94821D0E94B91D90E0909353
:100E0000FB018093FA01C23080E5D80721F480917C
:100E1000FA01816086C0C43090E5D90721F4809141
:100E2000FA0182607EC0C63020E5D20721F48091AD
:100E3000FA01846076C0C83080E5D80719F4809143
:100E4000FA0127C0CA3090E5D90721F48091FA0150
:100E5000806167C0CC3020E5D20721F48091FA018F
:100E600080625FC0CE3080E5D80721F48091FA011E
:100E7000806457C0C03190E5D90721F48091FA0110
:100E800080684FC0C23120E5D20729F48091FA0171
:100E90008460886046C0C33080E5D80721F4809123
:100EA000FA018E7F3EC0C53090E5D90721F48091CC
:100EB000FA018D7F36C0C73020E5D20721F480913A
:100EC000FA018B7F2EC0C93080E5D80719F48091D4
:100ED000FA0126C0CB3090E5D90721F48091FA01C0
:100EE0008F7E1FC0CD3020E5D20721F48091FA011A
:100EF0008F7D17C0CF3080E5D80721F48091FA01AB
:100F00008F7B0FC0C13190E5D90721F48091FA01A0
:100F10008F7707C0C331D04531F48091FA018B7FC0
:100F2000877F8093FA018091FA010E94BD1DABC0BA
:100F30008D2F99278F70992781309105D9F49E01C3
:100F40002370332702C0880F991F2A95E2F79C6807
:100F50008E0144E0000F111F4A95E1F7002713703E
:100F6000802B912B53E0CC0FDD1F5A95E1F7C07613
:100F7000DD272FC08230910531F4DC2FCC278E0184
:100F8000016F106A80C08330910569F4CE018370CF
:100F9000992701E010E002C0000F111F8A95E2F7C7
:100FA000C8019C680FC084309105B9F4CE018370EC
:100FB000992701E010E002C0000F111F8A95E2F7A7
:100FC000C8019A6823E0CC0FDD1F2A95E1F7C07EA7
:100FD000D7708C010C2B1D2B56C08530910531F438
:100FE000DC2FCC278E01046F106A4DC0069709F0E4
:100FF0004AC0CF71DD27DC2FCC278E01106243C0A1
:1010000000E010E040C08E013EC001E810E43BC0AB
:1010100003E810E438C002EE14E435C009EE14E42D
:1010200032C00AEE14E42FC005EB14E42CC006EB2A
:1010300014E429C007EB14E426C00CEC14E423C02C
:101040000DEC14E420C003E815E41DC00AE815E423
:101050001AC002E915E417C004E915E414C001E25E
:1010600016E411C003E216E40EC004E216E40BC05D
:1010700005E216E408C006E216E405C007E216E43D
:1010800002C00AE216E4C801DF91CF911F910F91CF
:10109000089596E0799FF001112494E5899FE00D71
:1010A000F11D1124E60FF11DEE0FFF1FE05FFE4F53
:1010B00085919491803E9105E0F4803C910558F52E
:1010C0008133910509F46FC048F48932910509F420
:1010D00063C08A32910509F46DC072C089339105ED
:1010E000E9F082389105D1F08533910509F44DC0BE
:1010F00067C0833E910581F138F4803E9105B9F0D7
:10110000823E9105D9F05CC0863E910561F1873E33
:101110009105A1F155C00E94060608952091FA019B
:1011200020FD02C021FF4CC080EE90E049C08091BC
:10113000FA0180FFF9CF89E390E042C08091FA0183
:1011400082FF0EC08091FA0184FF03C080E090E02E
:1011500037C083EE90E034C08091FA0182FFF2CF75
:1011600082EE90E02DC08091FA0183FF0BC0809148
:10117000FA0184FDEBCF87EE90E022C08091FA0166
:1011800083FFF5CF86EE90E01BC08091FA0185FFCA
:1011900007C089E290E014C08091FA0185FFF9CF81
:1011A00085E390E00DC08091FA0186FF07C08AE2D6
:1011B00090E006C08091FA0186FFF9CF81E390E0CC
:1011C0000E941606089508950C94E30880916E011C
:1011D0000895CF93DF9300D01F92CDB7DEB79C0167
:1011E0008091F101843019F593E099833B832A8340
:1011F0009093E9008FEF9091E800815095FD06C033
:1012000095ED9A95F1F700008111F5CF8091E800F6
:1012100085FF0DC040E050E063E070E0CE01019634
:101220000E94530B8091E8008E778093E8000F9026
:101230000F900F90DF91CF910895CF93DF9300D05F
:101240001F92CDB7DEB72091F101243021F522E0C5
:1012500029839B838A8383E08093E9008FEF9091B9
:10126000E800815095FD06C095ED9A95F1F70000D4
:101270008111F5CF8091E80085FF0DC040E050E07E
:1012800063E070E0CE0101960E94530B8091E8006C
:101290008E778093E8000F900F900F90DF91CF91A1
:1012A00008952091F1012430F1F422E02093E90027
:1012B0002FEF3091E800215035FD06C035ED3A950D
:1012C000F1F700002111F5CF2091E80025FF0BC0B8
:1012D00040E050E065E070E00E94530B8091E80030
:1012E0008E778093E8000895CF93DF93EC0190917F
:1012F000F101943009F046C080910C018823D9F0A7
:1013000080910D018823B9F09093E9008FEF9091BF
:10131000E800815095FD06C095E19A95F1F700002F
:101320008111F5CF8091E80085FF2CC040E050E0AE
:1013300060E170E017C081E08093E9008FEF909149
:10134000E800815095FD06C095ED9A95F1F70000F3
:101350008111F5CF8091E80085FF14C040E050E096
:1013600068E070E0CE010E94530B8091E8008E7718
:101370008093E80080E1FE01AEE5B1E001900D92BE
:101380008A95E1F7DF91CF9108958091F001811165
:1013900009C00E94E80C0E94450D8091E200846023
:1013A0008093E20008951092F001089508950C943E
:1013B0002C220E948D1B0E9432220E94EB0F0C9463
:1013C000E40842E061EC81E00E94620C42E061ECE2
:1013D00082E00E94620C42E061EC83E00E94620CB9
:1013E00042E161EC84E00C94620C8091F301833063
:1013F00009F455C030F4813071F0823009F48EC0A8
:1014000008958A3009F47AC08B3009F460C08930BD
:1014100009F09CC020C08091F201813A09F096C089
:101420008091E800877F8093E8008091F601909199
:10143000F701892B21F460E18EE591E003C060E0C3
:1014400080E090E070E00E949E0B8091E8008B7736
:101450008093E80008958091F201813209F076C00E
:101460008091F6019091F701009719F0039709F028
:101470006DC08091E800877F8093E8008091E8004C
:1014800082FD05C08091F1018111F8CF5FC080918C
:10149000F10080936E018091E8008B7753C08091BA
:1014A000F201813A09F052C08091F6019091F70162
:1014B000892B09F04BC08091E800877F8093E8007A
:1014C0008091E80080FFFCCF80910C0136C08091B4
:1014D000F2018132D9F58091F6019091F701892BC3
:1014E000A9F58091E800877F8093E8000E94970C1F
:1014F0008091F40180930C010C9484148091F2018A
:10150000813221F58091E800877F8093E8000E9476
:10151000970C8091F50180936F0108958091F201FD
:10152000813AA1F48091E800877F8093E800809160
:10153000E80080FFFCCF80916F018093F1008091E3
:10154000E8008E778093E8000C94970C089584B798
:10155000877F84BF88E10FB6F89480936000109273
:1015600060000FBE90E080E80FB6F89480936100B1
:10157000909361000FBE0E943A100E94E80C0E94F6
:10158000450D8091E20084608093E20078940E948F
:10159000CB0F0E943C1082E091E00E94E60F0E9477
:1015A0001A228091F101853069F40E94541B8091C8
:1015B000EF018823B1F30E947F1B882391F30E94DF
:1015C0003D0BEFCF0E944210ECCF292F3327233061
:1015D0003105C9F064F42130310581F02230310544
:1015E00009F043C08DE690E02CE333E042C02132A5
:1015F0003105F1F02232310541F137C082E190E04E
:1016000029EA33E036C099278130910541F08230D4
:10161000910541F0892B49F5E8E3F3E005C0E0E2EC
:10162000F3E002C0E8E0F3E0849190E09F0121C084
:101630006430D8F4E62FF0E0EE0FFF1FEE5DFE4FB2
:101640002081318189E090E014C0643070F470E052
:10165000FB01EE0FFF1FE65EFE4F20813181FB0193
:10166000EA5EFE4F808190E004C080E090E020E0E0
:1016700030E0FA0131832083089580E189BD82E161
:1016800089BD09B400FEFDCF8091D8008F7D809385
:10169000D8008091E00082608093E0008091E000BB
:1016A00081FDFCCF0895CF92DF92EF92FF920F93CE
:1016B0001F93CF93DF93EC018B016A010E94B60C5C
:1016C000811133C0C114D10439F0F60180819181B8
:1016D000081B190BC80FD91FE12CF12C011511059E
:1016E00019F18091E80085FD16C08091E8008E77A1
:1016F0008093E800C114D10449F0F6018081918102
:10170000E80EF91EF182E08285E00FC00E94B60C5F
:10171000882321F30AC089918093F10001501109B7
:10172000FFEFEF1AFF0ADACF80E0DF91CF911F9130
:101730000F91FF90EF90DF90CF9008952091F801E6
:101740003091F9012617370748F06115710539F412
:101750002091E8002E772093E80001C0B90140E015
:1017600061157105A9F12091F101222309F443C00B
:10177000253009F442C02091E80023FD40C02091AB
:10178000E80022FD32C02091E80020FFE9CF40911F
:10179000F3002091F20030E0342BFC01CF01611501
:1017A000710559F02830310540F481918093F100A2
:1017B000615071092F5F3F4FF1CF41E02830310573
:1017C00009F040E02091E8002E772093E800C8CF90
:1017D0004111C9CF0AC08091F101882361F08530A1
:1017E00061F08091E80083FD0AC08091E80082FFEB
:1017F000F2CF80E0089582E0089583E0089581E0CB
:1018000008952091F8013091F9012617370748F023
:101810006115710539F42091E8002E772093E800D6
:1018200001C0B901FC0120E06115710591F18091C1
:10183000F101882309F440C0853009F43FC080914C
:10184000E80083FD3DC08091E80082FD2FC08091BB
:10185000E80080FFE9CF2091F3008091F20090E052
:10186000922B6115710559F08830910540F424914F
:101870002093F1003196615071090196F2CF21E079
:10188000089709F020E08091E8008E778093E800C7
:10189000CBCF2111CCCF0AC08091F101882361F018
:1018A000853061F08091E80083FD0AC08091E800F6
:1018B00082FFF2CF80E0089582E0089583E00895EA
:1018C00081E00895982F973058F59093E900981784
:1018D00039F07091EC002091ED005091F00003C0C0
:1018E000242F762F50E021FF19C03091EB003E7F6E
:1018F0003093EB003091ED003D7F3093ED0030915F
:10190000EB0031603093EB007093EC002093ED001E
:101910005093F0002091EE0027FF07C09F5FD3CFC8
:101920008F708093E90081E0089580E008958091B0
:10193000F20187FF11C08091E80082FD05C080910F
:10194000F1018111F8CF11C08091E8008B770BC0B5
:101950008091F101882349F08091E80080FFF8CF61
:101960008091E8008E778093E80008952091E4004C
:101970003091E50095E64091EC00842F817040FFA6
:1019800022C08091E80080FD1CC08091F101882375
:1019900091F0853091F08091EB0085FD10C0409171
:1019A000E4005091E5004217530729F39A01915042
:1019B00011F784E0089582E0089583E0089581E0BE
:1019C000089580E008954091E80042FFDECF089539
:1019D0000E94560D0E945E0DE0EEF0E08081816075
:1019E0008083E8EDF0E080818F77808319BCA7EDDC
:1019F000B0E08C918E7F8C9380818F7E808310925B
:101A0000F00108950F931F93CF93DF930E94560D1B
:101A10000E945E0DC8EDD0E088818F778883888131
:101A20008068888388818F7D888319BC1092F1013A
:101A30001092ED011092EF011092EE0100EE10E015
:101A4000F80180818B7F808388818160888342E078
:101A500060E080E00E94620CE1EEF0E080818E7F29
:101A60008083E2EEF0E08081816080838081886005
:101A70008083F80180818E7F808388818061888364
:101A8000DF91CF911F910F910895E8EDF0E08081F3
:101A90008F7E8083E7EDF0E080818160808384E049
:101AA00082BF81E08093F0010C94020DE8EDF0E03C
:101AB00080818E7F80831092E20008951092DA0078
:101AC0001092E10008951F920F920FB60F92112409
:101AD0002F933F934F935F936F937F938F939F9336
:101AE000AF93BF93EF93FF938091E10082FF0BC010
:101AF0008091E20082FF07C08091E1008B7F80939C
:101B0000E1000E94CA0F8091DA0080FF1FC080911F
:101B1000D80080FF1BC08091DA008E7F8093DA00AE
:101B20008091D90080FF0DC080E189BD82E189BD2F
:101B300009B400FEFDCF81E08093F1010E94C50948
:101B400005C019BC1092F1010E94D3098091E100F7
:101B500080FF19C08091E20080FF15C08091E200F3
:101B60008E7F8093E2008091E20080618093E200AA
:101B70008091D80080628093D80019BC85E0809362
:101B8000F1010E94D7098091E10084FF30C080916B
:101B9000E20084FF2CC080E189BD82E189BD09B4E7
:101BA00000FEFDCF8091D8008F7D8093D80080917A
:101BB000E1008F7E8093E1008091E2008F7E809330
:101BC000E2008091E20081608093E2008091ED016B
:101BD000882311F084E007C08091E30087FD02C0F4
:101BE00081E001C083E08093F1010E94D9098091D6
:101BF000E10083FF29C08091E20083FF25C080912E
:101C0000E100877F8093E10082E08093F1011092F0
:101C1000ED018091E1008E7F8093E1008091E200F0
:101C20008E7F8093E2008091E20080618093E200E9
:101C300042E060E080E00E94620C8091F0008860E9
:101C40008093F0000E94D609FF91EF91BF91AF9170
:101C50009F918F917F916F915F914F913F912F91C4
:101C60000F900FBE0F901F9018951F920F920FB6F6
:101C70000F9211242F933F934F935F936F937F9312
:101C80008F939F93AF93BF93CF93DF93EF93FF9384
:101C9000C091E900CF708091EC00D82FD17080FD09
:101CA000D0E81092E9008091F000877F8093F000E7
:101CB00078940E94790E1092E9008091F00088607B
:101CC0008093F000CD2BCF70C093E900FF91EF918E
:101CD000DF91CF91BF91AF919F918F917F916F9144
:101CE0005F914F913F912F910F900FBE0F901F90DA
:101CF00018951F93CF93DF93CDB7DEB7AA970FB692
:101D0000F894DEBF0FBECDBFE2EFF1E088E08E0FAA
:101D10009091F10091938E13FBCF0E94F509809171
:101D2000E80083FF1FC18091F2019091F301492FD8
:101D300050E04A30510508F015C1FA01EA5AFF4F48
:101D40000C94B423803881F0823809F00BC1809163
:101D5000F6018F708093E9008091EB0085FB882766
:101D600080F91092E90006C08091EE019091EF0198
:101D7000911182609091E800977F9093E8008093A2
:101D8000F1001092F100C8C0282F2D7F09F0EAC0A1
:101D9000882319F0823061F0E5C08091F401813030
:101DA00009F0E0C0933009F080E08093EF012BC090
:101DB0008091F401811127C08091F6018F7009F4A0
:101DC000D1C08093E9002091EB0020FF1CC093302C
:101DD00021F48091EB00806214C09091EB0090613F
:101DE0009093EB0021E030E0A90102C0440F551FA1
:101DF0008A95E2F74093EA001092EA008091EB00A6
:101E000088608093EB001092E9008091E800877F62
:101E100086C08111A7C01091F4011F778091E30063
:101E20008078812B8093E3008091E800877F809306
:101E3000E8000E94970C8091E80080FFFCCF809121
:101E4000E30080688093E300111102C082E001C0CA
:101E500083E08093F10186C08058823008F082C010
:101E60008091F4019091F5018C3D53E0950779F54F
:101E700083E08A838AE289834FB7F894DE01139660
:101E800020E03EE051E2E32FF0E050935700E49170
:101E900020FF03C0E295EF703F5FEF708E2F90E060
:101EA000EA3010F0C79601C0C0968D939D932F5FC6
:101EB000243149F74FBF8091E800877F8093E80085
:101EC0006AE270E0CE0101960E949E0B14C0AE0142
:101ED0004F5F5F4F6091F6010E94E50ABC010097D9
:101EE00009F440C09091E800977F9093E8008981C1
:101EF0009A810E94010C8091E8008B778093E80022
:101F000031C0803879F58091E800877F8093E800C0
:101F10008091ED018093F1008091E8008E778093AD
:101F2000E8000E94970C1EC081111CC09091F40122
:101F30009230C0F48091E800877F8093E80090930E
:101F4000ED010E94970C8091ED01811106C08091F6
:101F5000E30087FD02C081E001C084E08093F101CD
:101F60000E94E1098091E80083FF0AC08091E800A7
:101F7000877F8093E8008091EB0080628093EB0084
:101F8000AA960FB6F894DEBF0FBECDBFDF91CF91FA
:101F90001F9108950895CF938091F1018823A1F0B6
:101FA000C091E900CF709091EC00892F817090FD75
:101FB00080E8C82B1092E9008091E80083FD0E9420
:101FC000790ECF70C093E900CF9108959093750179
:101FD000809374010895E0917401F0917501309738
:101FE00021F00190F081E02D099480E00895E091C6
:101FF0007401F0917501309721F00280F381E02D9A
:1020000009940895E0917401F0917501309721F0E1
:102010000480F581E02D099408952091720130919A
:1020200073018217930771F090937301809372018B
:10203000E0917401F0917501309721F00680F781ED
:10204000E02D09940895209170013091710182175B
:10205000930771F09093710180937001E091740186
:10206000F0917501309721F00084F185E02D0994FD
:10207000089508950C9439100E94931B0E94340314
:102080000C94551C9F92AF92BF92CF92DF92EF9229
:10209000FF920F931F93CF93DF9300D000D000D017
:1020A000CDB7DEB70E944C030DE010E0AA24A39444
:1020B000B12C902E802F0E943A04980129583E4F4F
:1020C0006901F901F080F826A1F40150110988F79F
:1020D0008FEF89838A831B820E949C1B8160782FEB
:1020E0009D838C8349815A816B818D810E94D91097
:1020F0002FC09091DA0191FF04C08E830E944004AA
:102100008E8125E030E0A501022E01C0440F0A9423
:10211000EAF7E42E4F21C1F029839A828E2191E0C3
:1021200009F490E09B830E949C1B8160782F9D8323
:102130008C8349815A816B818D810E94D910F6016F
:102140008081E826E08204C021503109E0F6BDCF4D
:102150000E943C1F109176010E94EB0F1817B9F0F6
:102160000E94EB0F8093760126960FB6F894DEBF9F
:102170000FBECDBFDF91CF911F910F91FF90EF90D8
:10218000DF90CF90BF90AF909F900C94E40826967C
:102190000FB6F894DEBF0FBECDBFDF91CF911F9178
:1021A0000F91FF90EF90DF90CF90BF90AF909F90F6
:1021B0000895CF93DF93CDB7DEB72B970FB6F89482
:1021C000DEBF0FBECDBF4F83588769877A878B8765
:1021D000DE01119686E0FD0111928A95E9F785E00E
:1021E000FE01379601900D928A95E1F749815A8157
:1021F0006B817C818D819E810E9422172B960FB668
:10220000F894DEBF0FBECDBFDF91CF910895CF937D
:10221000882309F4C2C0C82F823859F40E94EB0FFA
:1022200081FDBBC089E30E94FC190E94C91A89E3A1
:102230000CC0833879F40E94EB0F80FDAEC083E5BB
:102240000E94FC190E94C91A83E50E943E1ACF9190
:102250000C94C91A843859F40E94EB0F82FD9DC07A
:1022600087E40E94FC190E94C91A87E4EECF8CEF24
:102270008C0F813A48F48C2F0E947F2181118DC0F0
:102280008C2F0E94FC19E3CF80E28C0F883048F439
:10229000C77081E001C0880FCA95EAF70E94821AD0
:1022A000D6CF8BE58C0F833078F4C53A29F0C63A47
:1022B00031F083E890E005C081E890E002C082E858
:1022C00090E0CF910C940D1088E58C0F833108F0CD
:1022D00064C0C83A39F1C93A41F1CA3A49F1CB3A36
:1022E00051F1CC3A59F1CD3A61F1C03B69F1CE3AA6
:1022F00071F1CF3A79F1C13B81F1C23B89F1C33B26
:1023000091F1C43B99F1C53BA1F1C63BA9F1C73B93
:10231000B1F1C83BB9F1C93BC1F1CA3BC9F180E099
:1023200090E038C082EE90E035C089EE90E032C097
:102330008AEE90E02FC085EB90E02CC086EB90E019
:1023400029C087EB90E026C08CEC90E023C08DEC98
:1023500090E020C083E891E01DC08AE891E01AC0B7
:1023600082E991E017C084E991E014C081E292E033
:1023700011C083E292E00EC084E292E00BC085E2DD
:1023800092E008C086E292E005C087E292E002C0D7
:102390008AE292E0CF910C942310CF910895882384
:1023A00009F44BC0823859F40E94EB0F81FF45C0FD
:1023B00089E30E94FC190E94C91A89E30CC0833882
:1023C00071F40E94EB0F80FF38C083E50E94FC1976
:1023D0000E94C91A83E50E943E1A0C94C91A8438D7
:1023E00059F40E94EB0F82FF28C087E40E94FC1979
:1023F0000E94C91A87E4EFCF9CEF980F913A58F3E7
:1024000090E2980F983050F4877091E001C0990FD6
:102410008A95EAF7892F0E94881ADFCF9BE5980FEB
:10242000933020F480E090E00C940D10885A8331B2
:1024300020F480E090E00C9423100895882321F08C
:102440000E94821A0C94C91A0895882321F00E94D0
:10245000881A0C94C91A08957F928F929F92AF9216
:10246000BF92CF92DF92EF92FF920F931F93CF9381
:10247000DF931F92CDB7DEB77C01C62E772EFC010D
:10248000058102950F70128111110E949F1A0E94FE
:10249000F519882379F0112369F080E28C0D8830DA
:1024A00048F082E00E94DE190E94F51991E0D82ED2
:1024B000D92601C0D12CE72DE295EF70F0E0E05A6B
:1024C000FF4F0C94B423872D807F072D0F70882336
:1024D00011F00295007F112389F0002309F490C1C7
:1024E00080E28C0D883020F4802F0E94821A03C075
:1024F000802F0E94921A0E94C91A82C18C2D0E94BC
:10250000CF11002309F495C180E28C0D883020F4AE
:10251000802F0E94881A03C0802F0E94981A0E9460
:10252000C91A87C1972D907F872D8F70903211F037
:102530008295807FCC2021F0F1E0CF16B1F01EC053
:10254000112349F0002309F414C1013009F011C12D
:102550000E94B21A6EC1002319F0013009F469C15A
:1025600089830E94B51A89810AC1112321F00230A2
:1025700008F05FC1FEC001115CC101C1112321F04F
:10258000002309F4F6C03CC1002309F4F8C03EC1A1
:10259000872D86958695837090E0009719F00197B6
:1025A00061F047C1112321F08C2D972D937002C04B
:1025B00080E090E00E940D103CC1112321F08C2D91
:1025C000972D937002C080E090E00E94231031C1EB
:1025D0008C2D112319F00E94441E02C00E94AC1ED3
:1025E0000E94311F26C1872D837009F052C011113E
:1025F00020C18C2D829586958770880F880F9C2D21
:102600009F70892E912CA12CB12C082E04C0880C0F
:10261000991CAA1CBB1C0A94D2F7C4FE14C00FE07C
:1026200010E020E030E0B901A80104C0440F551FBC
:10263000661F771F8A95D2F7CB01BA016095709516
:102640008095909503C060E070E0CB01272D269522
:102650002695237030E02230310569F023303105B2
:1026600089F0682979298A299B292130310571F05F
:102670000E946A18DEC0682979298A299B290E944C
:102680008618D7C00E946A18C501B4010E944E186E
:10269000D0C0112319F0872D817001C08695882341
:1026A00009F4C7C08C2D829586958770880F880F96
:1026B0009C2D9F70892E912CA12CB12C082E04C02A
:1026C000880C991CAA1CBB1C0A94D2F7C4FE14C027
:1026D0000FE010E020E030E0B901A80104C0440F91
:1026E000551F661F771F8A95D2F7CB01BA016095F7
:1026F00070958095909503C060E070E0CB01272D28
:10270000269526952370422F50E04230510569F0FE
:102710004330510589F0682979298A299B2941305C
:10272000510571F00E94441984C0682979298A29C9
:102730009B290E9460197DC00E944419C501B40103
:102740000E94281976C08C2D90E0FC01E05EF10912
:10275000E531F10508F050C0E059FF4F0C94B42367
:102760000C2D0F70872D8F71112331F00E94C1182D
:10277000802F0E941E125DC00E94E218802F0E94CE
:10278000251257C0112339F0011153C0872D8F71C5
:102790000E9407194EC0023008F04BC0F7CF11233A
:1027A00039F0872D8F710E94C11843C01123C9F3DE
:1027B000872D8F710E94E2183CC0112329F0872DCC
:1027C0008F710E94AC1835C00E94A21832C011232C
:1027D00051F0172D1F71812F0E94C11863E0812FC6
:1027E0000E94D51926C081E00E94DE19023008F14E
:1027F00082E00E94DE191DC0112331F0002389F20E
:102800008C2D0E94071115C0002391F28C2D0E947F
:10281000CF110FC0472D4F706C2DC7010E941605B8
:102820000E94C61706C0472D4F706C2DC7010E942D
:10283000F305DD20F9F00E94D11980FD1BC0F701DE
:1028400012820E94CB190E94C118C7010E9449142C
:102850000E94CB190F90DF91CF911F910F91FF90A4
:10286000EF90DF90CF90BF90AF909F908F907F9030
:102870000C94E2180F90DF91CF911F910F91FF9070
:10288000EF90DF90CF90BF90AF909F908F907F9010
:1028900008950F931F93CF93DF93EC018881998163
:1028A0002B813C81232BB9F09F3F11F48F3F99F08E
:1028B000CE010E944B05882371F0688179818A815D
:1028C0000E94C7198C010E947C190E944318B8010C
:1028D000CE010E942C12DF91CF911F910F9108958C
:1028E0000E949F1A0E94AF1A0E94741A0E94C91A6D
:1028F0000E94E21F0E94311F80E090E00E940D10B4
:1029000080E090E00C9423100E948F1A0C947014B5
:102910000E94BC19292F22952F7030E02C303105F0
:102920004CF42A3031056CF4225031092230310543
:10293000A8F407C02C30310569F02F30310551F073
:102940000DC0803F69F018F4803E40F409C0843F18
:1029500029F406C093FB882780F9089580E0089544
:1029600081E00895CF93DF9300D000D01F92CDB7C0
:10297000DEB70F900F900F900F900F90DF91CF91D7
:102980000895CF93DF9300D000D000D0CDB7DEB74D
:1029900026960FB6F894DEBF0FBECDBFDF91CF9164
:1029A00008951F93CF93DF93C091850116E0809126
:1029B0008601C81799F0D0E01C9FF0011D9FF00D13
:1029C0001124E957FE4F40815181628173818481D6
:1029D00095810E94C1142196C770E9CFDF91CF91F4
:1029E0001F9108954091B7015091B8016091B901CC
:1029F0007091BA018091BB019091BC010C94C114FB
:102A00008091BC0182958F7009F054C08091B9010A
:102A1000882309F44FC080918501A09186016091BF
:102A2000B7017091B8014091BA015091BB01B6E075
:102A30008A1709F43FC090E041155105C1F17F3F6D
:102A400011F46F3FA1F1B89FF001B99FF00D11246F
:102A5000E957FE4F218172132AC02081621327C0DB
:102A60002281211124C0238134812417350710F4D9
:102A700021503109241B350B283C3105C0F420912D
:102A8000BC012F7020612093BC0126E0289FF0013B
:102A9000299FF00D1124E457FE4F80818F708061D3
:102AA000808387EB91E00E9449140C94D114019625
:102AB0008770BECF0895CF92DF92EF92FF920F936F
:102AC0001F93CF93DF93CDB7DEB762970FB6F8941D
:102AD000DEBF0FBECDBF8C0185E0F801DE011D9683
:102AE00001900D928A95E1F7D8014C9111965C9175
:102AF000119712966C9112971396CD90DC901497C3
:102B00003091B7017091B8018091BA019091BB01E9
:102B1000009709F46BC17F3F19F43F3F09F466C188
:102B2000E090B901EE2009F4C0C02091BC01C816A4
:102B3000D90628F0F601E81BF90BCF0104C08095F7
:102B400090958C0D9D1DFF24F394883C910578F0A1
:102B5000F12C207F09F0C6C07C2DD98AC88A8989CA
:102B60000E94B21487EB91E00E944914B1C0822FF9
:102B7000807F09F046C0751314C0341312C0611170
:102B800010C02F7020612093BC010E94F21487EBCB
:102B900091E00E9449148091BC01D80115968C9354
:102BA0002EC0CD2819F15F3F11F44F3FF9F0F62EFA
:102BB00061111CC0809185012091860136E0821749
:102BC00009F45AC090E0389FF001399FF00D1124AC
:102BD000E957FE4F7181571306C07081471303C038
:102BE0007281711103C001968770E9CFF62E6623BA
:102BF00009F418C18091BC0181608093BC01F12C63
:102C000011C1751308C0341306C0611104C080914E
:102C1000BC01D801C3C04D875E878D859E856A8BB8
:102C20000E9488146A898823E1F16623D1F12091FA
:102C3000BC01822F82958F7090E0029774F0809192
:102C4000B7019091B80198878F831986DB86CA8671
:102C50002C87CE0107960E94491486E0F801A7EB65
:102C6000B1E001900D928A95E1F70E9400150E9453
:102C7000F214FF24F394D6C04D875E878D859E8520
:102C80000E94BC19292F22952F7030E02230310587
:102C90000CF0BCC09F7009F0B6C0805E883008F4AC
:102CA000C1C0C8010E944914E4CFC816D90608F46F
:102CB00053C0F601E81BF90BCF01883C910508F4DD
:102CC00050C0F12C7C2DD98AC88A89890E94B214FF
:102CD000E7EBF1E086E0DF011D928A95E9F70E94BB
:102CE000F214A0C0751314C0341312C0611110C0C7
:102CF0008091BC01F8018583C8010E94491486E0D7
:102D0000E7EBF1E0DF011D928A95E9F7FE2C8AC01E
:102D10004D875E878D859E856A8B0E9488146A899F
:102D2000882309F4BECF662309F4BBCF2091BC01F0
:102D3000822F82958F7090E002970CF48ECF809155
:102D4000B7019091B8019A8389831B82DD82CC827E
:102D50002E83CE0101967FCF809590958C0D9D1D81
:102D6000ACCFF62E662309F49CCF75132EC0341316
:102D70002CC02091BC0120FD1FC0822F82958F7036
:102D8000D9F0D80115962C9315978F3049F08F5FA5
:102D9000982F9295907F822F8F70892B15968C9308
:102DA000C8010E94491486E0F801A7EBB1E0019048
:102DB0000D928A95E1F793CF86E0F801A7EBB1E099
:102DC00001900D928A95E1F72DC04D875E878D8524
:102DD0009E850E948814811140CF8091BC01816042
:102DE0008093BC01C8010E9449141CC0662309F4E9
:102DF00058CF4D875E878D859E850E9488148823D5
:102E000009F44FCF2ACF811148CF0CC024303105AF
:102E10000CF047CF9F7009F440CFF8019581907F67
:102E200009F03BCF8F2D62960FB6F894DEBF0FBE30
:102E3000CDBFDF91CF911F910F91FF90EF90DF9069
:102E4000CF9008951F93CF93DF93CDB7DEB72C9724
:102E50000FB6F894DEBF0FBECDBF4F83588769878A
:102E60007A878B879C87CE0107960E945B15882303
:102E700069F08F8198852A853B85232BF1F19F3F4F
:102E800009F063C08F3F09F060C037C086E0FE01E3
:102E90003796DE01119601900D928A95E1F76F81C8
:102EA0007885EA85FB85309741F17F3F11F46F3FCC
:102EB00021F12091860130E0C901019687709927A0
:102EC0004091850150E08417950709F447C0698354
:102ED0007A83FD83EC8396E0929FD001939FB00D9F
:102EE0001124A957BE4FFE01319601900D929A957B
:102EF000E1F7809386010E94D11416E0809185014C
:102F0000909186018917C1F1189FC001112489573A
:102F10009E4F0E945B15882379F1E09185011E9FE9
:102F2000F0011124E957FE4F408151816281738184
:102F3000848195810E94C1148091850190E0019661
:102F40008770992780938501D9CF4F8158856985EE
:102F50007A858B859C850E94C114CFCF0E948414F2
:102F60001092860110928501E7EBF1E086E0DF0127
:102F70001D928A95E9F7C1CF2C960FB6F894DEBF63
:102F80000FBECDBFDF91CF911F910895EF92FF92B9
:102F90000F931F93CF93DF938C01009709F46CC0BC
:102FA000F12CEE24E394E8012196F8018491843712
:102FB00040F4843008F051C0813081F0823019F142
:102FC0005BC0853709F444C0A8F19CE7980F90379F
:102FD00008F052C08F770E94CF1141C00E5F1F4F83
:102FE000FE01C49180E28C0F883048F4C7708E2DAA
:102FF00001C0880FCA95EAF70E94A21A14C08C2F4C
:103000000E9407112DC00E5F1F4FFE01C49180E288
:103010008C0F883058F4C7708E2D01C0880FCA9568
:10302000EAF70E94A81A0E94C91A1AC08C2F0E949F
:10303000CF1116C00E5F1F4FFE01C491CC2381F04B
:103040008FE99FE00197F1F700C00000C150F6CF73
:103050000E5F1F4FFE01F49003C00E9407118E0106
:103060008F2D882309F49FCFEFE9FFE03197F1F727
:1030700000C000008150F5CFDF91CF911F910F91DB
:10308000FF90EF90089508956093C1017093C2017D
:103090008093C3019093C4010C9470140F931F93F9
:1030A0000091C1011091C2012091C3013091C4016E
:1030B000DC01CB01802B912BA22BB32B8093C10180
:1030C0009093C201A093C301B093C4011F910F91CB
:1030D0000C9470140F931F930091C1011091C201C1
:1030E0002091C3013091C401DC01CB0180239123E5
:1030F000A223B3238093C1019093C201A093C30183
:10310000B093C4011F910F910C9470140F931F93EF
:103110000091C1011091C2012091C3013091C401FD
:10312000DC01CB0180279127A227B3278093C1011F
:103130009093C201A093C301B093C4011F910F915A
:103140000C9470141092BD011092BE011092BF0138
:103150001092C0010C94701441E050E060E070E007
:1031600004C0440F551F661F771F8A95D2F74093FE
:10317000BD015093BE016093BF017093C0010C94D8
:10318000701441E050E060E070E004C0440F551F4F
:10319000661F771F8A95D2F78091BD019091BE017D
:1031A000A091BF01B091C001482B592B6A2B7B2BFA
:1031B0004093BD015093BE016093BF017093C00165
:1031C0000C94701441E050E060E070E004C0440FE3
:1031D000551F661F771F8A95D2F7409550956095C9
:1031E00070958091BD019091BE01A091BF01B091F9
:1031F000C001482359236A237B234093BD01509388
:10320000BE016093BF017093C0010C94701441E043
:1032100050E060E070E004C0440F551F661F771F48
:103220008A95D2F78091BD019091BE01A091BF0116
:10323000B091C001482759276A277B274093BD01D9
:103240005093BE016093BF017093C0010C94701441
:103250000F931F930091BD011091BE012091BF01FA
:103260003091C001DC01CB01802B912BA22BB32B21
:103270008093BD019093BE01A093BF01B093C001A4
:103280001F910F910C9470140F931F930091BD0127
:103290001091BE012091BF013091C001DC01CB0132
:1032A00080239123A223B3238093BD019093BE0179
:1032B000A093BF01B093C0011F910F910C947014A3
:1032C0000F931F930091BD011091BE012091BF018A
:1032D0003091C001DC01CB0180279127A227B327C1
:1032E0008093BD019093BE01A093BF01B093C00134
:1032F0001F910F910C9470140895CF92DF92EF926A
:10330000FF920F931F93CF93DF938C01C090C10165
:10331000D090C201E090C301F090C4018091BD0142
:103320009091BE01A091BF01B091C001C82AD92AD5
:10333000EA2AFB2ACFE1D0E0D701C6010C2E04C057
:10334000B695A795979587950A94D2F780FF06C002
:10335000B8018C2F0E944908019721F4219760F74A
:1033600080E001C08C2FDF91CF911F910F91FF90D2
:10337000EF90DF90CF900895CF93DF93EC010E9400
:103380007D19BE010E944908DF91CF910895CB01BC
:103390000E94BC1908958091C501859585958595F4
:1033A00008958091C5018770089598E0899F9001E4
:1033B0001124262B2093C5010C94C1182091C5011E
:1033C000809582238093C501982F977069F430E02F
:1033D000482F552747FD50952417350729F0859527
:1033E000859585950C94E21808959091C501977084
:1033F00081E009F480E0089590910C01992321F077
:1034000090910D01911109C020910E0130910F0191
:10341000F90132969FEF40E01FC0982F9695969540
:1034200096959F3050F5E0910E01F0910F01E90F54
:10343000F11D877021E030E0A90102C0440F551F43
:103440008A95E2F7CA019181892B818308959F3F74
:1034500039F04F5F4E3041F051915813F8CF0DC005
:103460005111F7CF942FF5CF9F3F39F0F901E90FB4
:10347000F11D97FDFA9582830895089590910C01AE
:10348000992321F090910D01911109C020910E0115
:1034900030910F01F9013296205F3F4F1FC0982FE6
:1034A0009695969596959F30F0F4E0910E01F091E7
:1034B0000F01E90FF11D877021E030E0A90102C082
:1034C000440F551F8A95E2F7CA018095918189239F
:1034D000818308953196E217F30729F090819813BC
:1034E000F9CF1082F7CF089581E090E0E0910E01CE
:1034F000F0910F01E80FF91F1082019680319105BC
:10350000A9F708959091D901892B8093D901089545
:1035100080959091D90189238093D90108951092C3
:10352000D90108959091D801892B8093D8010895ED
:1035300080959091D80189238093D80108951092A5
:10354000D80108959091D701892B8093D7010895D0
:1035500080959091D70189238093D7010895109287
:10356000D70108958093C60108951092C601089569
:1035700080910E0190910F01FC0131969C01205F1A
:103580003F4F80E0919191118F5FE217F307D1F7E0
:103590000895E0910E01F0910F018091D90180838F
:1035A000E0910E01F0910F0190818091D801892B5B
:1035B0008083E0910E01F0910F0190818091D701FD
:1035C000892B80838091C601882361F0E0910E01F0
:1035D000F0910F019081892B80830E94B81A81118C
:1035E0001092C60180910E0190910F010C94F70F7B
:1035F00020E0009739F0AC01415051098423952314
:103600002F5FF7CF822F0895CF92DF92EF92FF9234
:103610006C01EE24FF24C114D104E104F10421F073
:10362000C701B60120E101C020E0C72ED82EE92E47
:10363000FF24C114D104E104F10419F0285FC7018B
:10364000B6016B017C0154E0F694E794D794C794DB
:103650005A95D1F7C114D104E104F10419F02C5F9B
:10366000C701B6016B017C0142E0F694E794D79460
:10367000C7944A95D1F7C114D104E104F10419F0BB
:103680002E5FC701B601DC01CB01B695A7959795D2
:103690008795892B8A2B8B2B09F02F5F822FFF9028
:1036A000EF90DF90CF9008958091F101843021F167
:1036B0001092DB0120E488E190E00FB6F894A89521
:1036C000809360000FBE2093600080E00E94E408B9
:1036D00083B7817F846083BF83B7816083BF789421
:1036E000889583B78E7F83BF88E10FB6F894809367
:1036F0006000109260000FBE0895089508950E9422
:103700007D1B0E944C030E947E1B0E94410491E09D
:10371000811101C090E0892F08950E9484140E94B5
:10372000EB0F0C94E40882E084BD93E095BD9AEF22
:1037300097BD80936E0008952FB7F8948091DC01B7
:103740009091DD01A091DE01B091DF012FBF0895BE
:10375000CF92DF92EF92FF920F931F932FB7F894BF
:103760004091DC015091DD016091DE017091DF013B
:103770002FBF6A017B01EE24FF248C0120E030E0A2
:10378000C016D106E206F30610F4415051099A0121
:10379000281B390BC9011F910F91FF90EF90DF900B
:1037A000CF9008951F920F920FB60F9211248F930E
:1037B0009F93AF93BF938091DC019091DD01A09125
:1037C000DE01B091DF010196A11DB11D8093DC01E6
:1037D0009093DD01A093DE01B093DF01BF91AF9123
:1037E0009F918F910F900FBE0F901F9018950E9480
:1037F000E80CF8942FEF87EA91E621508040904042
:10380000E1F700C0000087E090EBDC018093FB0152
:103810009093FC01A093FD01B093FE019CE088E130
:103820000FB6F894A895809360000FBE9093600047
:10383000FFCFEF92FF920F931F93CF93DF93D82F79
:10384000CDE08C2F0E943A0405E010E0E82EF12C28
:10385000C701002E02C0959587950A94E2F780FF74
:1038600009C0602F7C2F80E00E94F405D81302C0AD
:1038700081E006C00150110958F7C15010F780E0EF
:10388000DF91CF911F910F91FF90EF900895CF930B
:10389000C82F8CE20E94191C882321F08C2FCF9115
:1038A0000C94191C80E0CF910895CF930E949C1D29
:1038B000811102C00E94821DC5E6C15049F00E94DC
:1038C0004C038FE39CE90197F1F700C00000F5CFAE
:1038D00089E20E94471C811113C18AE20E94471CA1
:1038E00081110E94821D85E00E94471C81110E9467
:1038F000F71B0E94A71D8093DA0187E00E94471CF6
:103900008823A9F18BE10E94471C882351F0809104
:10391000DA0181FB222720F991E0922790FB81F9BF
:103920000EC08EE00E94471C882361F08091DA016E
:1039300082FB222720F991E0922790FB82F9809365
:10394000DA0115C080E10E94471C9091DA018823BA
:1039500041F093FB222720F981E0822780FB93F935
:1039600004C0892F809580FB90F99093DA018091B3
:10397000DA010E94AB1D0E94B91D8093FA0180EE0E
:103980000E94471C882341F08091FA01982F90955E
:1039900090FB80F98093FA0189E30E94471C8823F9
:1039A00059F08091FA0181FB222720F991E09227BA
:1039B00090FB81F98093FA0182EE0E94471C8823D4
:1039C00059F08091FA0182FB222720F991E0922799
:1039D00090FB82F98093FA0186EE0E94471C8823AF
:1039E00059F08091FA0183FB222720F991E0922778
:1039F00090FB83F98093FA0183EE0E94471C882391
:103A000059F08091FA0184FB222720F991E0922756
:103A100090FB84F98093FA0185E30E94471C882378
:103A200059F08091FA0185FB222720F991E0922735
:103A300090FB85F98093FA0181E30E94471C88235B
:103A400059F08091FA0186FB222720F991E0922714
:103A500090FB86F98093FA0181E10E94471C88233C
:103A600059F08091FA0187FB222720F991E09227F3
:103A700090FB87F98093FA018091FA010E94BD1DA5
:103A80008091FA0187FB882780F980930D0187E2F6
:103A90000E94471CC82F8EE10E94471C8111C26002
:103AA0008FE10E94471C8111C46080E20E94471C84
:103AB0008111C86081E20E94471C8111C06182E2CD
:103AC0000E94471C8111C06283E20E94471C811141
:103AD000C06484E20E94471C882311F0C06802C0C1
:103AE000CC2329F08C2F0E94B41D6C2F03C00E94A0
:103AF000B01D682F70E080E090E0CF910C944418E6
:103B0000CF9108956DEE7EEF80E090E00E94EE236D
:103B100060E082E090E00E94DC2360E083E090E0DF
:103B20000E94DC2360E084E090E00E94DC2360E0FF
:103B300085E090E00C94DC2380E090E00E94D623A6
:103B400021E08D3E9E4F09F020E0822F089582E013
:103B500090E00C94CE23682F82E090E00C94DC235C
:103B600083E090E00C94CE23682F83E090E00C94E7
:103B7000DC2384E090E00C94CE23682F84E090E076
:103B80000C94DC238091E20180FF0BC06091130153
:103B900085E0689FB00111247595679575956795C7
:103BA0002BC081FF09C06091130185E0689FB001BF
:103BB00011247595679520C082FF07C0609113019D
:103BC00085E0689FB001112417C09091E30199230B
:103BD000D1F060911201961788F72091130185E0CA
:103BE000289F90011124929FA001939F500D1124B2
:103BF00070E0CA010E94A0236038710540F461158D
:103C0000710539F002C065E070E0862F08958FE7F6
:103C1000089581E008958091E20180FF08C06091DD
:103C2000110170E0759567957595679521C081FFC5
:103C300006C06091110170E07595679519C082FF0B
:103C400004C06091110170E010C09091E3019923CC
:103C5000C1F0609110019617A0F780911101899F22
:103C6000C001112470E00E94A0236038710528F47F
:103C70006115710521F0862F08958FE7089581E081
:103C8000089561E070E0F4CF803F21F40E94C21DEE
:103C9000819504C0813F29F40E94C21D8093E601F2
:103CA0000895823F21F40E94C21D819504C0833F84
:103CB00029F40E94C21D8093E5010895893F19F4FB
:103CC0000E940B1E05C08A3F31F40E940B1E819595
:103CD0008093E70108958B3F21F40E940B1E81958C
:103CE00004C08C3F29F40E940B1E8093E8010895C4
:103CF000843F21F48091E401816017C0853F21F465
:103D00008091E401826011C0863F21F48091E4013A
:103D100084600BC0873F21F48091E401886005C076
:103D2000883F31F48091E40180618093E40108953B
:103D30008D3F21F48091E20181600BC08E3F21F420
:103D40008091E201826005C08F3F29F48091E201F9
:103D500084608093E2010895803F39F48091E60108
:103D600087FF6CC01092E60169C0813F29F4809101
:103D7000E6011816BCF362C09091E501823F29F478
:103D800097FF5CC01092E50159C0833F19F41916E2
:103D9000CCF354C0893F41F48091E70118160CF030
:103DA0004DC01092E7014AC08A3F29F48091E70193
:103DB00087FF44C0F6CF8B3F39F48091E80187FF3D
:103DC0003DC01092E8013AC08C3F29F48091E8018F
:103DD0001816BCF333C0843F21F48091E4018E7F38
:103DE00017C0853F21F48091E4018D7F11C0863F8B
:103DF00021F48091E4018B7F0BC0873F21F48091F7
:103E0000E401877F05C0883F31F48091E4018F7E13
:103E10008093E40113C08D3F21F48091E2018E7FF5
:103E20000BC08E3F21F48091E2018D7F05C08F3F52
:103E300029F48091E2018B7F8093E2018091E5017A
:103E400081110EC08091E60181110AC08091E701C5
:103E5000811106C08091E801811102C01092E30136
:103E6000089584EE91E00E9402100E949C1B9093A2
:103E7000E1018093E00108951F93CF93DF93809138
:103E8000E0019091E1010E94A81BAC019091E30137
:103E9000992321F02091140130E006C020911501F2
:103EA0008AE0289F900111244217530708F486C026
:103EB0008091E501C091E601D091E7011091E80100
:103EC000811107C0C11176C0D11174C0111172C027
:103ED00075C09F3F19F09F5F9093E301181624F47B
:103EE0000E94C21D8093E5018091E50187FF05C016
:103EF0000E94C21D81958093E5011C1624F40E9446
:103F0000C21D8093E6018091E60187FF05C00E94F3
:103F1000C21D81958093E6016091E501662339F128
:103F2000C091E601CC2319F1772767FD7095872FA3
:103F3000972F0E94B12223E333E343E35FE30E9420
:103F400015230E947E226093E5016C2F772767FD81
:103F50007095872F972F0E94B12223E333E343E329
:103F60005FE30E9415230E947E226093E6011D16E6
:103F700024F40E940B1E8093E7018091E70187FFE4
:103F800005C00E940B1E81958093E701111624F451
:103F90000E940B1E8093E8018091E80187FF05C015
:103FA0000E940B1E81958093E801DF91CF911F91B4
:103FB0000C94311F9F3F09F08ECF96CFDF91CF91A8
:103FC0001F910895E4EEF1E085E0DF011D928A95EE
:103FD000E9F71092E3011092E2010895833081F134
:103FE00028F4813059F08230D1F00895853009F4F9
:103FF00049C0B8F1863009F456C008958091150182
:10400000262F30E0280F311D2F3F310524F4680F93
:104010006093150108958FEF8093150108958091A5
:104020001401262F30E0280F311D2F3F310524F4D5
:10403000680F6093140108958FEF80931401089521
:1040400080911301262F30E0280F311D2F3F3105BD
:1040500024F4680F6093130108958FEF8093130188
:10406000089580911201262F30E0280F311D2F3F37
:10407000310524F4680F6093120108958FEF809347
:104080001201089580911101262F30E0280F311D73
:104090002F3F310524F4680F6093110108958FEFCD
:1040A00080931101089580911001262F30E0280F90
:1040B000311D2F3F310524F4680F609310010895DE
:1040C0008FEF809310010895833011F128F481302F
:1040D00049F0823091F00895853081F120F18630E9
:1040E000C1F1089580911501681720F4861B809313
:1040F0001501089510921501089580911401681713
:1041000020F4861B809314010895109214010895E1
:1041100080911301681720F4861B80931301089582
:1041200010921301089580911201681720F4861BE4
:104130008093120108951092120108958091110147
:10414000681720F4861B80931101089510921101C5
:10415000089580911001681720F4861B8093100148
:1041600008951092100108950F931F938D3109F453
:104170006BC008F03FC08E3009F47FC0C0F48730B8
:1041800009F469C068F4863009F0B1C08091DA01A1
:10419000817F8E7F8093DA0181E08093EA01A8C05D
:1041A000883009F4A2C08B3009F49FC0A0C08631CA
:1041B00009F49BC078F4803109F472C0813109F0B0
:1041C00096C00E94841490910D0181E0892780930C
:1041D0000D018BC0893109F488C08B3109F087C08B
:1041E0008091DA0181FB222720F991E0922790FB50
:1041F00081F94CC0853309F470C048F4873209F462
:104200006CC008F459C0893209F467C070C08334A7
:1042100038F48A3308F04EC0883309F466C067C0AA
:10422000833409F45AC0883409F061C00E948414B0
:104230000FEF13ED20E3015010402040E1F700C0E4
:1042400000000E94F71B51C00E9438220E94EB0F11
:104250000E94E4084AC09091DA01892F809581700C
:1042600080FB90F929F0966098609093DA0140C045
:10427000997F977F9093DA0138C08091DA0182FBB1
:10428000222720F991E0922790FB82F98093DA01AE
:10429000992359F18091DA0181608093DA0125C078
:1042A0008091DA0183FB222720F991E0922790FB8D
:1042B00083F9ECCF895301C08D5141E050E060E0BB
:1042C00070E08A019B0104C0000F111F221F331FE1
:1042D0008A95D2F7C901B80104C061E070E080E0BE
:1042E00090E00E9444180E94841481E001C080E0A4
:1042F0001F910F91089580E0089580E00895CF9375
:10430000C82F8091EA01813079F018F08230E9F10C
:1043100087C0E0910E01F0910F018081813169F039
:10432000823209F07FC009C0E0910E01F0910F01C7
:104330008081813111F0823261F48C2F0E947B21C7
:10434000811104C08C2F0E94B4201DC081E090E038
:104350001AC08C2F0E947D21811114C0C43179F0C4
:1043600048F4CB3079F0C03109F060C082E080932E
:10437000EA0108C0C93219F0C83321F057C01092C1
:10438000EA0154C081E0817053C0C93289F118F547
:10439000C43171F1A8F4C73009F046C08AE08093B7
:1043A000150194E19093140193E09093130180938D
:1043B000120188E08093110188E28093100134C0DB
:1043C000CE51C63088F5EC2FF0E0E65DFE4F8081DF
:1043D0008093E90129C0CE34E9F020F4CB3421F5F3
:1043E0006AE013C0C13579F0C235F1F461E00DC067
:1043F0008091E901882319F01092E90115C081E04C
:104400008093EA0115C061E006C08091E9010E9435
:10441000EE1F0AC06AE08091E9010E94642004C096
:104420001092EA0180E004C081E002C080E0ABCFDE
:10443000CF910895E1E8F0E08081886080838081F9
:10444000816080838FB7F89493E09093890090ED1A
:10445000909388008FBF0895EFE6F0E0808182603E
:1044600080830895EFE6F0E080818D7F808308955A
:10447000EFE6F0E0908182E08927808308951F9223
:104480000F920FB60F9211242F933F934F935F9388
:104490006F937F938F939F93AF93BF93EF93FF930C
:1044A0008091EB019091EC0101969093EC01809347
:1044B000EB01811103C082E00E94E408E091EC016D
:1044C000E695E695F0E0EA54FB4FE4918091EB012C
:1044D0008E1303C080E00E94E408FF91EF91BF912A
:1044E000AF919F918F917F916F915F914F913F918C
:1044F0002F910F900FBE0F901F90189504D06894C5
:10450000B1118DC0089570D088F09F5790F0B92FE9
:104510009927B751A0F0D1F0660F771F881F991F18
:104520001AF0BA95C9F712C0B13081F077D0B1E076
:10453000089574C0672F782F8827B85F39F0B93F86
:10454000CCF3869577956795B395D9F73EF490951A
:104550008095709561957F4F8F4F9F4F0895E89498
:1045600009C097FB3EF490958095709561957F4FBB
:104570008F4F9F4F9923A9F0F92F96E9BB27939569
:10458000F695879577956795B795F111F8CFFAF479
:10459000BB0F11F460FF1BC06F5F7F4F8F4F9F4FAA
:1045A00016C0882311F096E911C0772321F09EE808
:1045B000872F762F05C0662371F096E8862F70E06E
:1045C00060E02AF09A95660F771F881FDAF7880F48
:1045D0009695879597F9089557FD9058440F551F64
:1045E00059F05F3F71F04795880F97FB991F61F075
:1045F0009F3F79F087950895121613061406551FEC
:10460000F2CF4695F1DF08C0161617061806991F57
:10461000F1CF86957105610508940895E894BB274C
:1046200066277727CB0197F908950BD078C069D01A
:1046300028F06ED018F0952309F05AC05FC01124FD
:10464000EECFCADFA0F3959FD1F3950F50E0551F31
:10465000629FF001729FBB27F00DB11D639FAA27D7
:10466000F00DB11DAA1F649F6627B00DA11D661F26
:10467000829F2227B00DA11D621F739FB00DA11D47
:10468000621F839FA00D611D221F749F3327A00D01
:10469000611D231F849F600D211D822F762F6A2F9D
:1046A00011249F5750408AF0E1F088234AF0EE0F22
:1046B000FF1FBB1F661F771F881F91505040A9F72F
:1046C0009E3F510570F014C0AACF5F3FECF3983EB7
:1046D000DCF3869577956795B795F795E7959F5F96
:1046E000C1F7FE2B880F911D9695879597F9089530
:1046F00097F99F6780E870E060E008959FEF80EC95
:10470000089500240A941616170618060906089537
:1047100000240A9412161306140605060895092E9D
:104720000394000C11F4882352F0BB0F40F4BF2B0C
:1047300011F460FF04C06F5F7F4F8F4F9F4F08954C
:1047400097FB072E16F4009407D077FD09D00E943E
:10475000BA2307FC05D03EF4909581959F4F0895AC
:10476000709561957F4F0895EE0FFF1F0590F491AE
:10477000E02D0994AA1BBB1B51E107C0AA1FBB1F58
:10478000A617B70710F0A61BB70B881F991F5A95DD
:10479000A9F780959095BC01CD010895F999FECFB8
:1047A00092BD81BDF89A992780B50895A8E1B0E03F
:1047B00042E050E00C94F623262FF999FECF92BDEB
:1047C00081BDF89A019700B4021639F01FBA20BDD6
:1047D0000FB6F894FA9AF99A0FBE08950196272F0A
:1047E0000E94DD230C94DC23DC01CB01FC01F99950
:1047F000FECF06C0F2BDE1BDF89A319600B40D922D
:0C48000041505040B8F70895F894FFCFE5
:10480C000220E608740951091D09E9080101C701D4
:10481C0028080A03140A3F4D363977042A04F40396
:10482C00BB034E03670380039903010203040506CF
:04483C000708090060
:00000001FF
